Microchip MPLAB XC8 Compiler V2.36

Linker command line:

-W-3 --edf=/opt/microchip/xc8/v2.36/pic/dat/en_msgs.txt -cn \
  -h+dist/default/production/UART_TX_18F452_2.X.production.sym \
  --cmf=dist/default/production/UART_TX_18F452_2.X.production.cmf -z \
  -Q18F452 -o/tmp/xcXCjofjM --defsym=__MPLAB_BUILD=1 \
  -Mdist/default/production/UART_TX_18F452_2.X.production.map \
  --md=/tmp/xcXGnKJdH.dat -E1 -ver=XC8 Compiler --acfsm=1493 \
  -ACODE=00h-03FFFhx2 -ACONST=00h-07FFFh -ASMALLCONST=0600h-06FFhx122 \
  -AMEDIUMCONST=0600h-07FFFh -ACOMRAM=01h-07Fh -AABS1=00h-05FFh \
  -ABIGRAM=01h-05FFh -ARAM=080h-0FFh,0100h-01FFhx5 -ABANK0=080h-0FFh \
  -ABANK1=0100h-01FFh -ABANK2=0200h-02FFh -ABANK3=0300h-03FFh \
  -ABANK4=0400h-04FFh -ABANK5=0500h-05FFh -ASFR=0F80h-0FFFh \
  -ABIGSFR=0F80h-0FFFh -ACONFIG=0300000h-030000Dh -AIDLOC=0200000h-0200007h \
  -AEEDATA=0F00000h-0F000FFh -peeprom_data=EEDATA \
  -preset_vec=00h,intcode=08h,intcodelo,powerup,init -pramtop=0600h \
  -psmallconst=SMALLCONST -pmediumconst=MEDIUMCONST -pconst=CONST \
  -AFARRAM=00h-00h \
  -prdata=COMRAM,nvrram=COMRAM,nvbit=COMRAM,rbss=COMRAM,rbit=COMRAM \
  -pfarbss=FARRAM,fardata=FARRAM,nvFARRAM=FARRAM \
  -pintsave_regs=BIGRAM,bigbss=BIGRAM,bigdata=BIGRAM -pbss=RAM \
  -pidata=CODE,irdata=CODE,ibigdata=CODE,ifardata=CODE -prparam=COMRAM \
  /tmp/xcXHoHeNI.o dist/default/production/UART_TX_18F452_2.X.production.o 

Object code version is 3.11

Machine type is 18F452



                Name                               Link     Load   Length Selector   Space Scale
/tmp/xcXHoHeNI.o
                idloc                            200000   200000        8        0       5
                config                           300000   300000        E        0       4
                text                                A42      A42        2      302       0
                init                                 B2       B2        4        4       0
                reset_vec                             0        0        6        0       0
dist/default/production/UART_TX_18F452_2.X.production.o
                intcode                               8        8       AA        4       0
                idloc                            200000   200000        8        0       5
                config                           300000   300000        E        0       4
                temp                                 3E       3E        1        1       1
                smallconst                          600      600        4      300       0
                text19                              854      854       48      302       0
                text17                              8E2      8E2       34      302       0
                text16                              A26      A26        C      302       0
                text15                              A1A      A1A        C      302       0
                text14                              916      916       26      302       0
                text13                              99C      99C       1E      302       0
                text12                              93C      93C       24      302       0
                text11                              97E      97E       1E      302       0
                text10                              78C      78C       7C      302       0
                text9                               960      960       1E      302       0
                text8                               6FE      6FE       8E      302       0
                text7                               9F0      9F0       1A      302       0
                text6                               604      604       FA      302       0
                text5                               A0A      A0A       10      302       0
                text4                               A3A      A3A        8      302       0
                text3                               A32      A32        8      302       0
                text2                               9BA      9BA       1C      302       0
                text1                               9D6      9D6       1A      302       0
                text0                               89C      89C       46      302       0
                cstackCOMRAM                         23       23       19        1       1
                bssBANK1                            100      100       FF      100       1
                bssBANK0                             80       80       64       80       1
                dataCOMRAM                           3D       3D        1        1       1
                bssCOMRAM                             1        1       22        1       1
                cinit                               808      808       4C      302       0
                nvCOMRAM                             3C       3C        1        1       1
                idataCOMRAM                         A44      A44        1      302       0

TOTAL           Name                               Link     Load   Length     Space
        CLASS   CODE           
                intcode                               8        8       AA         0
                text                                A42      A42        2         0
                init                                 B2       B2        4         0
                reset_vec                             0        0        6         0
                text19                              854      854       48         0
                text17                              8E2      8E2       34         0
                text16                              A26      A26        C         0
                text15                              A1A      A1A        C         0
                text14                              916      916       26         0
                text13                              99C      99C       1E         0
                text12                              93C      93C       24         0
                text11                              97E      97E       1E         0
                text10                              78C      78C       7C         0
                text9                               960      960       1E         0
                text8                               6FE      6FE       8E         0
                text7                               9F0      9F0       1A         0
                text6                               604      604       FA         0
                text5                               A0A      A0A       10         0
                text4                               A3A      A3A        8         0
                text3                               A32      A32        8         0
                text2                               9BA      9BA       1C         0
                text1                               9D6      9D6       1A         0
                text0                               89C      89C       46         0
                cinit                               808      808       4C         0
                idataCOMRAM                         A44      A44        1         0

        CLASS   CONST          

        CLASS   SMALLCONST     
                smallconst                          600      600        4         0

        CLASS   MEDIUMCONST    

        CLASS   COMRAM         
                temp                                 3E       3E        1         1
                cstackCOMRAM                         23       23       19         1
                dataCOMRAM                           3D       3D        1         1
                bssCOMRAM                             1        1       22         1
                nvCOMRAM                             3C       3C        1         1

        CLASS   ABS1           

        CLASS   BIGRAM         

        CLASS   RAM            

        CLASS   BANK0          
                bssBANK0                             80       80       64         1

        CLASS   BANK1          
                bssBANK1                            100      100       FF         1

        CLASS   BANK2          

        CLASS   BANK3          

        CLASS   BANK4          

        CLASS   BANK5          

        CLASS   SFR            

        CLASS   BIGSFR         

        CLASS   CONFIG         
                config                           300000   300000        E         4

        CLASS   IDLOC          
                idloc                            200000   200000        8         5

        CLASS   EEDATA         

        CLASS   FARRAM         

        CLASS   HEAP           

        CLASS   STACK          



SEGMENTS        Name                           Load    Length   Top    Selector   Space  Class

                bssCOMRAM                      000001  00003E  00003F         1       1  COMRAM  
                reset_vec                      000000  000006  000006         0       0  CODE    
                text6                          000604  000441  000A45       302       0  CODE    
                bssBANK0                       000080  000064  0000E4        80       1  BANK0   
                bssBANK1                       000100  0000FF  0001FF       100       1  BANK1   
                intcode                        000008  0000AE  0000B6         4       0  CODE    
                smallconst                     000600  000004  000604       300       0  SMALLCON


UNUSED ADDRESS RANGES

        Name                Unused          Largest block    Delta
        BANK0            0000E4-0000FF               1C
        BANK1            0001FF-0001FF                1
        BANK2            000200-0002FF              100
        BANK3            000300-0003FF              100
        BANK4            000400-0004FF              100
        BANK5            000500-0005FF              100
        BIGRAM           00003F-00007F               41
                         0000E4-0000FF               1C
                         0001FF-0005FF              401
        BIGSFR           000F80-000FFF               80
        CODE             000006-000007                2
                         0000B6-0005FF              54A
                         000A45-007FFF             35BB
        COMRAM           00003F-00007F               41
        CONST            000006-000007                2
                         0000B6-0005FF              54A
                         000A45-007FFF             75BB
        EEDATA           F00000-F000FF              100
        MEDIUMCONST      000A45-007FFF             75BB
        RAM              0000E4-0000FF               1C
                         0001FF-0005FF              100
        SFR              000F80-000FFF               80
        SMALLCONST       000A45-007FFF              100

                                  Symbol Table

I2C_Master_Write@data                                                  cstackCOMRAM 000032
IO_Expander_Write@Data                                                 cstackCOMRAM 000033
LCD_CMD@CMD                                                            cstackCOMRAM 000035
LCD_Init@I2C_Add                                                       cstackCOMRAM 000038
LCD_Set_Cursor@COL                                                     cstackCOMRAM 000036
LCD_Set_Cursor@ROW                                                     cstackCOMRAM 000039
LCD_Write_4Bit@Nibble                                                  cstackCOMRAM 000034
LCD_Write_Char@Data                                                    cstackCOMRAM 000035
LCD_Write_String@Str                                                   cstackCOMRAM 000036
LCD_Write_String@i                                                     cstackCOMRAM 00003A
_ACKDT                                                                 (abs)        007E2D
_ACKEN                                                                 (abs)        007E2C
_ACKSTAT                                                               (abs)        007E2E
_BackLight_State                                                       dataCOMRAM   00003D
_I2C_Master_Init                                                       text7        0009F0
_I2C_Master_Start                                                      text16       000A26
_I2C_Master_Stop                                                       text15       000A1A
_I2C_Master_Wait                                                       text17       0008E2
_I2C_Master_Write                                                      text14       000916
_INTCONbits                                                            (abs)        000FF2
_IO_Expander_Write                                                     text13       00099C
_LATDbits                                                              (abs)        000F8C
_LCD_CMD                                                               text11       00097E
_LCD_Init                                                              text6        000604
_LCD_Set_Cursor                                                        text10       00078C
_LCD_Write_4Bit                                                        text12       00093C
_LCD_Write_Char                                                        text9        000960
_LCD_Write_String                                                      text8        0006FE
_PEN                                                                   (abs)        007E2A
_PIE1bits                                                              (abs)        000F9D
_PIR1bits                                                              (abs)        000F9E
_RCEN                                                                  (abs)        007E2B
_RCONbits                                                              (abs)        000FD0
_RCREG                                                                 (abs)        000FAE
_RCSTAbits                                                             (abs)        000FAB
_RS                                                                    bssCOMRAM    000022
_RSEN                                                                  (abs)        007E29
_SEN                                                                   (abs)        007E28
_SPBRG                                                                 (abs)        000FAF
_SSPADD                                                                (abs)        000FC8
_SSPBUF                                                                (abs)        000FC9
_SSPCON1                                                               (abs)        000FC6
_SSPCON2                                                               (abs)        000FC5
_SSPIF                                                                 (abs)        007CF3
_SSPSTAT                                                               (abs)        000FC7
_TRISC3                                                                (abs)        007CA3
_TRISC4                                                                (abs)        007CA4
_TRISC6                                                                (abs)        007CA6
_TRISC7                                                                (abs)        007CA7
_TRISDbits                                                             (abs)        000F95
_TXREG                                                                 (abs)        000FAD
_TXSTAbits                                                             (abs)        000FAC
__HRAM                                                                 (abs)        000000
__Habs1                                                                abs1         000000
__Hbank0                                                               bank0        000000
__Hbank1                                                               bank1        000000
__Hbank2                                                               bank2        000000
__Hbank3                                                               bank3        000000
__Hbank4                                                               bank4        000000
__Hbank5                                                               bank5        000000
__Hbigbss                                                              bigbss       000000
__Hbigdata                                                             bigdata      000000
__Hbigram                                                              bigram       000000
__Hbigsfr                                                              bigsfr       000000
__Hbss                                                                 bss          000000
__HbssBANK0                                                            bssBANK0     000000
__HbssBANK1                                                            bssBANK1     000000
__HbssCOMRAM                                                           bssCOMRAM    000000
__Hcinit                                                               cinit        000000
__Hclrtext                                                             clrtext      000000
__Hcomram                                                              comram       000000
__Hconfig                                                              config       30000E
__Hconst                                                               const        000000
__HcstackCOMRAM                                                        cstackCOMRAM 000000
__Hdata                                                                data         000000
__HdataCOMRAM                                                          dataCOMRAM   000000
__Heeprom_data                                                         eeprom_data  000000
__Hfarbss                                                              farbss       000000
__Hfardata                                                             fardata      000000
__Hheap                                                                heap         000000
__Hibigdata                                                            ibigdata     000000
__Hidata                                                               idata        000000
__HidataCOMRAM                                                         idataCOMRAM  000000
__Hidloc                                                               idloc        200008
__Hifardata                                                            ifardata     000000
__Hinit                                                                init         0000B6
__Hintcode                                                             intcode      0000B2
__Hintcode_body                                                        intcode_body 000000
__Hintcodelo                                                           intcodelo    0000B2
__Hintentry                                                            intentry     000000
__Hintret                                                              intret       000000
__Hintsave_regs                                                        intsave_regs 000000
__Hirdata                                                              irdata       000000
__Hmediumconst                                                         mediumconst  000000
__HnvCOMRAM                                                            nvCOMRAM     000000
__HnvFARRAM                                                            nvFARRAM     000000
__Hnvbit                                                               nvbit        000000
__Hnvrram                                                              nvrram       000000
__Hparam                                                               rparam       000000
__Hpowerup                                                             powerup      0000B2
__Hram                                                                 ram          000000
__Hramtop                                                              ramtop       000600
__Hrbit                                                                rbit         000000
__Hrbss                                                                rbss         000000
__Hrdata                                                               rdata        000000
__Hreset_vec                                                           reset_vec    000006
__Hrparam                                                              rparam       000000
__Hsfr                                                                 sfr          000000
__Hsmallconst                                                          smallconst   000604
__Hspace_0                                                             (abs)        000A45
__Hspace_1                                                             (abs)        0001FF
__Hspace_2                                                             (abs)        000000
__Hspace_4                                                             (abs)        60000E
__Hstack                                                               stack        000000
__Hstruct                                                              struct       000000
__Htemp                                                                temp         00003F
__Htext                                                                text         000000
__Htext0                                                               text0        000000
__Htext1                                                               text1        000000
__Htext10                                                              text10       000000
__Htext11                                                              text11       000000
__Htext12                                                              text12       000000
__Htext13                                                              text13       000000
__Htext14                                                              text14       000000
__Htext15                                                              text15       000000
__Htext16                                                              text16       000000
__Htext17                                                              text17       000000
__Htext19                                                              text19       000000
__Htext2                                                               text2        000000
__Htext3                                                               text3        000000
__Htext4                                                               text4        000000
__Htext5                                                               text5        000000
__Htext6                                                               text6        000000
__Htext7                                                               text7        000000
__Htext8                                                               text8        000000
__Htext9                                                               text9        000000
__LRAM                                                                 (abs)        000001
__Labs1                                                                abs1         000000
__Lbank0                                                               bank0        000000
__Lbank1                                                               bank1        000000
__Lbank2                                                               bank2        000000
__Lbank3                                                               bank3        000000
__Lbank4                                                               bank4        000000
__Lbank5                                                               bank5        000000
__Lbigbss                                                              bigbss       000000
__Lbigdata                                                             bigdata      000000
__Lbigram                                                              bigram       000000
__Lbigsfr                                                              bigsfr       000000
__Lbss                                                                 bss          000000
__LbssBANK0                                                            bssBANK0     000000
__LbssBANK1                                                            bssBANK1     000000
__LbssCOMRAM                                                           bssCOMRAM    000000
__Lcinit                                                               cinit        000000
__Lclrtext                                                             clrtext      000000
__Lcomram                                                              comram       000000
__Lconfig                                                              config       000000
__Lconst                                                               const        000000
__LcstackCOMRAM                                                        cstackCOMRAM 000000
__Ldata                                                                data         000000
__LdataCOMRAM                                                          dataCOMRAM   000000
__Leeprom_data                                                         eeprom_data  000000
__Lfarbss                                                              farbss       000000
__Lfardata                                                             fardata      000000
__Lheap                                                                heap         000000
__Libigdata                                                            ibigdata     000000
__Lidata                                                               idata        000000
__LidataCOMRAM                                                         idataCOMRAM  000000
__Lidloc                                                               idloc        000000
__Lifardata                                                            ifardata     000000
__Linit                                                                init         0000B2
__Lintcode                                                             intcode      000008
__Lintcode_body                                                        intcode_body 000000
__Lintcodelo                                                           intcodelo    0000B2
__Lintentry                                                            intentry     000000
__Lintret                                                              intret       000000
__Lintsave_regs                                                        intsave_regs 000000
__Lirdata                                                              irdata       000000
__Lmediumconst                                                         mediumconst  000000
__LnvCOMRAM                                                            nvCOMRAM     000000
__LnvFARRAM                                                            nvFARRAM     000000
__Lnvbit                                                               nvbit        000000
__Lnvrram                                                              nvrram       000000
__Lparam                                                               rparam       000000
__Lpowerup                                                             powerup      0000B2
__Lram                                                                 ram          000000
__Lramtop                                                              ramtop       000600
__Lrbit                                                                rbit         000000
__Lrbss                                                                rbss         000000
__Lrdata                                                               rdata        000000
__Lreset_vec                                                           reset_vec    000000
__Lrparam                                                              rparam       000000
__Lsfr                                                                 sfr          000000
__Lsmallconst                                                          smallconst   000600
__Lspace_0                                                             (abs)        000000
__Lspace_1                                                             (abs)        000000
__Lspace_2                                                             (abs)        000000
__Lspace_4                                                             (abs)        000000
__Lstack                                                               stack        000000
__Lstruct                                                              struct       000000
__Ltemp                                                                temp         00003E
__Ltext                                                                text         000000
__Ltext0                                                               text0        000000
__Ltext1                                                               text1        000000
__Ltext10                                                              text10       000000
__Ltext11                                                              text11       000000
__Ltext12                                                              text12       000000
__Ltext13                                                              text13       000000
__Ltext14                                                              text14       000000
__Ltext15                                                              text15       000000
__Ltext16                                                              text16       000000
__Ltext17                                                              text17       000000
__Ltext19                                                              text19       000000
__Ltext2                                                               text2        000000
__Ltext3                                                               text3        000000
__Ltext4                                                               text4        000000
__Ltext5                                                               text5        000000
__Ltext6                                                               text6        000000
__Ltext7                                                               text7        000000
__Ltext8                                                               text8        000000
__Ltext9                                                               text9        000000
__S0                                                                   (abs)        000A45
__S1                                                                   (abs)        0001FF
__S4                                                                   (abs)        000000
__S5                                                                   (abs)        000000
___heap_hi                                                             (abs)        000000
___heap_lo                                                             (abs)        000000
___inthi_sp                                                            stack        000000
___intlo_sp                                                            stack        000000
___param_bank                                                          (abs)        000000
___rparam_used                                                         (abs)        000001
___sp                                                                  stack        000000
__accesstop                                                            (abs)        000080
__activetblptr                                                         (abs)        000002
__cntErrataNOP_/tmp/xcXHoHeNI.o                                        (abs)        000001
__cntErrataNOP_dist/default/production/UART_TX_18F452_2.X.production.o (abs)        000046
__end_of_I2C_Master_Init                                               text7        000A0A
__end_of_I2C_Master_Start                                              text16       000A32
__end_of_I2C_Master_Stop                                               text15       000A26
__end_of_I2C_Master_Wait                                               text17       000916
__end_of_I2C_Master_Write                                              text14       00093C
__end_of_IO_Expander_Write                                             text13       0009BA
__end_of_LCD_CMD                                                       text11       00099C
__end_of_LCD_Init                                                      text6        0006FE
__end_of_LCD_Set_Cursor                                                text10       000808
__end_of_LCD_Write_4Bit                                                text12       000960
__end_of_LCD_Write_Char                                                text9        00097E
__end_of_LCD_Write_String                                              text8        00078C
__end_of__initialization                                               cinit        000846
__end_of_adint                                                         intcode      0000B2
__end_of_boot                                                          text1        0009F0
__end_of_init_interrupts                                               text5        000A1A
__end_of_init_uart                                                     text2        0009D6
__end_of_main                                                          text0        0008E2
__end_of_rx_start                                                      text4        000A42
__end_of_strcpy                                                        text19       00089C
__end_of_tx_start                                                      text3        000A3A
__initialization                                                       cinit        000808
__mediumconst                                                          mediumconst  000000
__pbssBANK0                                                            bssBANK0     000080
__pbssBANK1                                                            bssBANK1     000100
__pbssCOMRAM                                                           bssCOMRAM    000001
__pcinit                                                               cinit        000808
__pcstackCOMRAM                                                        cstackCOMRAM 000023
__pdataCOMRAM                                                          dataCOMRAM   00003D
__pidataCOMRAM                                                         idataCOMRAM  000A44
__pintcode                                                             intcode      000008
__pnvCOMRAM                                                            nvCOMRAM     00003C
__psmallconst                                                          smallconst   000600
__ptext0                                                               text0        00089C
__ptext1                                                               text1        0009D6
__ptext10                                                              text10       00078C
__ptext11                                                              text11       00097E
__ptext12                                                              text12       00093C
__ptext13                                                              text13       00099C
__ptext14                                                              text14       000916
__ptext15                                                              text15       000A1A
__ptext16                                                              text16       000A26
__ptext17                                                              text17       0008E2
__ptext19                                                              text19       000854
__ptext2                                                               text2        0009BA
__ptext3                                                               text3        000A32
__ptext4                                                               text4        000A3A
__ptext5                                                               text5        000A0A
__ptext6                                                               text6        000604
__ptext7                                                               text7        0009F0
__ptext8                                                               text8        0006FE
__ptext9                                                               text9        000960
__ramtop                                                               ramtop       000600
__smallconst                                                           smallconst   000600
_adint                                                                 intcode      000008
_boot                                                                  text1        0009D6
_cont_rc                                                               bssCOMRAM    00001F
_data                                                                  bssCOMRAM    000021
_i2c_add                                                               nvCOMRAM     00003C
_init_interrupts                                                       text5        000A0A
_init_uart                                                             text2        0009BA
_main                                                                  text0        00089C
_rc_buff                                                               bssBANK0     000080
_rc_data                                                               bssBANK1     000100
_rx_start                                                              text4        000A3A
_strcpy                                                                text19       000854
_test_buff                                                             bssCOMRAM    000001
_tx_start                                                              text3        000A32
btemp                                                                  temp         00003E
end_of_initialization                                                  cinit        000846
int$flags                                                              temp         00003E
intlevel0                                                              text         000A42
intlevel1                                                              text         000A42
intlevel2                                                              text         000A42
intlevel3                                                              text         000A42
isa$std                                                                (abs)        000001
isa$xinst                                                              (abs)        000000
stackhi                                                                (abs)        000000
stacklo                                                                (abs)        000000
start                                                                  init         0000B2
start_initialization                                                   cinit        000808
strcpy@d                                                               cstackCOMRAM 000029
strcpy@dest                                                            cstackCOMRAM 000023
strcpy@s                                                               cstackCOMRAM 000027
strcpy@src                                                             cstackCOMRAM 000025
ttemp5                                                                 temp         00003F
ttemp6                                                                 temp         000042
ttemp7                                                                 temp         000046
wtemp8                                                                 temp         00003F


MODULE INFORMATION

Module		Function		Class		Link	Load	Size
lcd_i2c.c
		_LCD_Init      		CODE           	0604	0000	250
		_LCD_Write_4Bit		CODE           	093C	0000	36
		_LCD_Write_Char		CODE           	0960	0000	30
		_LCD_CMD       		CODE           	097E	0000	30
		_I2C_Master_Wait		CODE           	08E2	0000	52
		_I2C_Master_Init		CODE           	09F0	0000	26
		_I2C_Master_Stop		CODE           	0A1A	0000	12
		_LCD_Set_Cursor		CODE           	078C	0000	124
		_IO_Expander_Write		CODE           	099C	0000	30
		_I2C_Master_Write		CODE           	0916	0000	38
		_I2C_Master_Start		CODE           	0A26	0000	12
		_LCD_Write_String		CODE           	06FE	0000	142

lcd_i2c.c estimated size: 782

mainTx.c
		_adint         		CODE           	0008	0000	170
		_boot          		CODE           	09D6	0000	26
		_main          		CODE           	089C	0000	70
		_init_uart     		CODE           	09BA	0000	28
		_rx_start      		CODE           	0A3A	0000	8
		_tx_start      		CODE           	0A32	0000	8
		_init_interrupts		CODE           	0A0A	0000	16

mainTx.c estimated size: 326

shared
		__initialization		CODE           	0808	0000	62

shared estimated size: 62

/opt/microchip/xc8/v2.36/pic/sources/c99/common/strcpy.c
		_strcpy        		CODE           	0854	0000	72

/opt/microchip/xc8/v2.36/pic/sources/c99/common/strcpy.c estimated size: 72

